:020000040000FA
:060000000219FD0200B32D
:03002B0002008D43
:03005B0002028717
:030073000200A0E8
:100080000406080C10182030406080A0C0C0D0C00A
:10009000E0C2CF0541E52360021523D0E0D0D03285
:1000A000C2AF53E67F7592FA7593FFC22053917FDA
:1000B000D2AF32C0D0C0E0C0F0D2D35388EFA88A0C
:1000C000A98C758A00758C0043881030331FE8C4F2
:1000D000540FFAE9C454F04AFAC3132AFAC3E833B6
:1000E000F8E933F9E82AFAE93403FB213630320F14
:1000F000C3E833E933FAE82AFAE93400FB21363061
:100100003115E875F056A4AAF0E975F056A42AFA5C
:10011000C5F03400FB2136E875F02BA4AAF0E97590
:10012000F02BA42AFAC5F03400C313FBEA13FAC378
:10013000EB13FBEA13FAC3EB94095006C3EB9403E9
:10014000501A0522E52270021522C3E522940A50B6
:1001500002417D7552007A007B00414EE52260022B
:1001600015223035067C007D042176AC31AD32306D
:100170003A04AC33AD34C3EA9CFAEB9DFB9208AE73
:100180005EAF5F303A425007203409D234219430B8
:100190003402C234303404AE60AF61203902B2346C
:1001A000C3EA33FAEB33FBA208500AEAF42401FA5B
:1001B000EBF43400FBC3EA9428FAEB9400FB5014F0
:1001C00078007A007B0021D4A208500878007A00D9
:1001D0007B00412AE52554036019202A16E55BF9C6
:1001E000EB7007C3E99A4002E9FAE53CC42AFAEB4E
:1001F0003400FBEA8EF0A4F9AAF0EB8EF0A42AFA00
:10020000C5F03400FBC3EB13FDEA13F80FEF1460E5
:1002100004C3E833F8C3E933EA33FAEB33FBDFED29
:10022000EB30E20678FF7AFF7B038852D230C3E8D6
:1002300094404002D221C3E559FC955A4003AC5A80
:10024000C3EC95525008EC75F004A4FAABF0EAF454
:10025000F8EBF45403F9C3E89414FAE99400FB5062
:10026000047A007B00885489558A568B5775230A77
:10027000D0F0D0E0D0D053F7DF43F7403275230AF7
:10028000D0F0D0E0D0D032C0D0C0E0D2D3A8F9E5D1
:100290005830E007E5FA30E10741D5E5FA30E135BD
:1002A000C3E55513F8E55413F5FB88FCC3E5571374
:1002B000F8E55613F5E988EA85555853F7BFC3E5C5
:1002C000529401400575530041D5E5532401F5537F
:1002D00050037553FF53F7DFD0E0D0D0327901805F
:1002E0001479038010790A800C791E800879648063
:1002F0000479C880007817E4D5E0FDD8FAD9F62251
:100300007A147B7880127A107B8C800C7A0D7BB407
:1003100080067A0B7BC880007902E4C291D5E0FDAB
:10032000D290D5E0FDC290D5E0FDD291D5E0FDE9B7
:1003300020E002D28630E002D292E562D5E0FDE90B
:1003400020E002C28630E002C2927496D5E0FDD968
:10035000C9EAF8D5E0FDD8FBDBBEC2912278FFC226
:100360002120283D202912D221C3E548940A4009C2
:10037000C3E55294405002C22179A1E76023E548C9
:10038000601F74FF8548F084853FF030290375F0C5
:1003900005A4F8C5F0600278FFC3E8955B5002A899
:1003A0005B885A22C3E54794E4E5489400E55A5037
:1003B000031461B5046002F55A2275E89022055CC9
:1003C000C3E55C94084055E5E820ECF2A8BDA9BE61
:1003D000755C00E9FA79A0E76041EA7006E55D60C6
:1003E00018800CC3E8955D600EE55D5005600A1449
:1003F00080070460FA8002E55DF55DC394F6401B5A
:100400007559C0C394064013755980C39406400BB8
:10041000755940C39406400375590022E5592410CC
:10042000500274FFF55922743279A687F0A4C5F002
:10043000A2F733F8C3E895594002A859885B2275A2
:1004400047007548F022C2AF75C800A8CCA9CDAA54
:100450004130CF010A75C804D2AFAB42AC438842E9
:100460008943C3E89BF8E99C202808F9302C02A1B5
:100470005281AFAD448A44F9EA9DFA600478FF796D
:10048000FFAE45AF468B458C46A842A943C3E89EC4
:10049000F8E99FF9C3E54813FBE54713FAE82AF5A5
:1004A00047E93BF54850067547FF7548FF81F9AAB3
:1004B00047AB48AC47AD487E047F02C3EB94044091
:1004C0000A1E1FC3EB940840021E1FC3ED13FDEC70
:1004D00013FCDEF7C3EA9CFAEB9DFBEF6009C3E96E
:1004E00013F9E813F8DFF7EA28FAEB39FB8A478BB0
:1004F0004850067BFF8B478B48C3EB94025002D2D7
:100500002C3028047F03A1247892E6FFC3E53D94B4
:100510008240110FC3E53D94A040010FC3EF940644
:1005200040027F057E02E548C4540FF9E548C454F3
:10053000F0F8E547C4540F28F8C3E89EFAE99400A0
:10054000FB4009C3EA9401EB940050047A01E4FBF8
:10055000A19EAA47AB48EBC4FEEAC4540F4EFCC3AD
:10056000EA9CFAEB9400FBC3E813C313F8EA28FAF9
:10057000EB3400FB8A478B48C3EB94024002C22C49
:100580007802EBC4FE7B00EAC4540F4EFAC3EA982B
:10059000FA4005C3940150027A017892E6FF3020B8
:1005A0000280FB854E92854F93D22043E680C3E4C0
:1005B0009AF8E49BF9302C02C129E8FAE9FBD3E967
:1005C00013FDE813FC884E894FC3EF94036037EFA7
:1005D00020E00CE82CF8E93DF9ECFAEDFB8013E89B
:1005E00028F8E939F9C3E82401F8E93400F97AFF79
:1005F0007BFFC3EF9403400E8A508B51884A894B8E
:100600008C4C8D4DC15D885089518A4A8B4B8C4CE6
:100610008D4D3028127550F07551FF754CF0754DA9
:10062000FF754EF0754FFFC15DE8FAD3E813FC8803
:100630004EC3EF94036020EF20E007E82CF8ECFABB
:10064000C149E8282401F87AFFC3EF940340088ADF
:1006500050884A8C4CC15D88508A4A8C4C302002AC
:10066000C15D753A02D22043E680E525540360342B
:10067000A847A948C3E913F9E813F8C3E913F9E84F
:1006800013F8302804E92440F9C2AF53E67F75918E
:1006900000C3E498F594E499F595759104D220434C
:1006A000E680D2AF22D222754900752000302B039C
:1006B000752040800ED222754900752040302B03F2
:1006C00075200078017901202C20E5255403600273
:1006D000C2227914E548C313700104F8C39414408E
:1006E000027814302804781B791B202010E549601B
:1006F0000C302803D53A04D224E165D1650549E5DB
:100700009B5440B52002E14F30280908C3E89940C6
:100710000118C1EA20220A08C3E8994002C1C3C1F6
:10072000EAC222C2AF53E67F759100302C12759455
:10073000007595FE759104D22043E680D2AFC1C307
:10074000AE47AF48C3E49EF594E49FF595E134C30A
:10075000E53994015002C1C3302202C1C3D802E17D
:1007600063C1EAC224C2AF53E67F759100855094FD
:10077000855195759104854A92854B93D22043E625
:1007800080D2AFE525540360072029020539801087
:1007900030240D202B0A20220715811581020E9B83
:1007A0002278003021053022027801E53D75F007FE
:1007B000A4F9E5F028F5F0E9A2F013A2F113A2F2F2
:1007C00013F53DC394785003753D78C3E53D953EE0
:1007D000400ED223C286C290C29275D4FF75D50F47
:1007E00030200280FB854C92854D93D22043E680D9
:1007F00022203813C2AFC291D28775D4FF75D503BA
:10080000D2AF759F4201E9C2AFC291D29375D43F76
:1008100075D50FD2AF759F4201E9203814C2AFC21F
:100820009275D4FF75D50CD287D2AF759F5202084E
:10083000E9C2AFC28675D4FF75D50CD293D2AF751D
:100840009F320208E9203813C2AFC287D29375D411
:10085000FF75D50CD2AF759F3201E9C2AFC293D2FA
:100860008775D4FF75D50CD2AF759F52807B203829
:1008700014C2AFC29075D43F75D50FD293D2AF7565
:100880009F420208E9C2AFC29075D4FF75D503D26A
:1008900087D2AF759F420208E9203813C2AFC293D6
:1008A000D29175D43F75D50FD2AF759F52803AC2A1
:1008B000AFC287D29175D4FF75D503D2AF759F3281
:1008C0008027203813C2AFC28675D4FF75D503D2F6
:1008D00091D2AF759F328011C2AFC29275D43F756D
:1008E000D50FD291D2AF759F52C22322C286C29039
:1008F000C292C287C291C29375D4FF75D50F227878
:100900008076FF0876FF0876FF0876FF0876FF08F6
:1009100076FF0876090876FF087601788C7601085C
:1009200076FF0876FF0876FF0876FF0876FF0876E0
:10093000030876FF0876FF0876FF0876250876D04C
:100940000876280876500876040876FF08760208AC
:1009500076FF08767A0876FF087601087601087631
:10096000FF0876FF08760008760022FA75F00CA4DE
:10097000ABF0EAC333F8740133F9E8C333F8E93371
:10098000F9E8C32BF8E93400F9227888E6C3940328
:10099000D23A5002C23AC238E630E102D238A23826
:1009A00092397886E6149000809378A6F67886E6E9
:1009B000F53FC394025003753F02789CE6753EFFF5
:1009C000B40203753EA0B40303753E827896E63107
:1009D0006B88318932789EE6316B88338934789719
:1009E000E6316B8835893611EC223035117A007B7F
:1009F000007CFF7D007E0051518B5F8A5E22303A81
:100A0000227896E6FA7B00789EE6FC7D00C3EA3306
:100A1000FAEB33FBC3EC33FCED33FD7E0A51518B13
:100A2000618A607896303A02789EE6FA7B00789781
:100A3000E6FC7D007E00303A10C3EA33FAEB33FB6C
:100A4000C3EC33FCED33FD7E0A51518B5F8A5E228D
:100A500022C3EC9EFCED9400FDC3EC9AFCED9BFDE3
:100A6000C3EC9423ED940050047C237D00C3EC94EC
:100A7000FFED940140047CFF7D017BFF0B7A000AAF
:100A8000EA7009C3EC33FCED33FD417CEC8AF0A441
:100A9000AEF0ED8AF0A42E947C40E4EAF460DD220E
:100AA000D23531EA1202E97A007B007C101202E1B1
:100AB000E5522AFA74003BFBDCF37C04C3EB13FB26
:100AC000EA13FADCF7FFEB60027FFFC23531EA225E
:100AD00078A5E6F954037000E9540C7000E954302D
:100AE0007000E954C0700022E5EF20E60375200095
:100AF0000520903FFFE520146006901DFF14600064
:100B00009304600375EF127597DE7597AD7581C01C
:100B100043FF801202DD75EF0275A90011EC7580AC
:100B20003F75F1C375A4C075803F75D4FF75900003
:100B300075F20F75A50F75900075D50F75A6017527
:100B4000E34075E20211ECE4F8F6D8FD11FFD1CDD7
:100B500078988662753001C2AF1202F1120300125A
:100B600002E91203061202E912030C1202E951D043
:100B7000C2AF78FA79FA308007D9FBD8F7021C00A7
:100B8000318A31EA7898866211EC75E40075881133
:100B9000758E0475890975C80475910475D84075FA
:100BA000D90875F781759E0375960275DA4275DB73
:100BB0004275A82175E69075F310759B80759D00B0
:100BC00075D12C75BC5875BB1075E88075B20112D3
:100BD00002DDD2AF753C00C2301202F1C231752283
:100BE000001202EDC3E522940A4024D231C23275CC
:100BF00022001202EDC3E522940A4013D232C2331E
:100C00007522001202EDC3E522940A4002D233128B
:100C100002E1203003020B70C2AF12030012030086
:100C2000120300D2AF1202F1303A0281BA1202E18D
:100C3000788CE6C39401500281BAE530C394015028
:100C40000281BA7F02D23531EA1202EDC2AFC2355B
:100C500031EAAE52C3E552947FD2AF405D1202DD5D
:100C6000C2AF120312D2AFDFDC51A0C3EF7897F608
:100C70001202F1F107F1A97F0AD23531EA1202ED31
:100C8000C2AFC23531EAAE52C3E552947FD2AF5003
:100C9000E61202DDC2AF1203001202E5120300D217
:100CA000AFDFD651A0EF24037896F61202F1F107D8
:100CB000120FD81202ED31EA61701202ED780130A4
:100CC0003A027805C3E5529840028128C2AF120368
:100CD00012120312120312D2AF1202F1753000E4A5
:100CE000F537F5380537E537F4703E0538789AE67C
:100CF0007819146012783214600D787D14600878C9
:100D0000FA146003753800C3E53898401C11EC12E2
:100D100002DD153875370078998662C2AF1203126A
:100D2000D2AF789886621202ED1202E5E5237002D6
:100D300061707801C3E5529840AA1202EDE5237074
:100D400003020B70C2AF11ECE4D2AFE4F55CF52402
:100D5000F525F53D755C081202DD1203BAE5E820C1
:100D6000ECFBA8BDA9BEE97001F8885D1203BE7551
:100D70005C08C2AF7559FF120427855B59855B5A21
:100D8000D2AF303A07C238303402D238D22875395F
:100D900000119911C212043F12044612043F1204BA
:100DA0004612043F1206B51207A11207F1120446BB
:100DB0001206A5202C0312035D302C031203A4128B
:100DC00007A1111A1204461206B51207A111451205
:100DD00004461206A51207A1116E1204461206B5AA
:100DE0001207A111991204461203BA1206A512079E
:100DF000A111C21203BE120446302827855B59791F
:100E0000187A0CC3E53999400EC228D2298A3B854D
:100E10005B59855B5A800CC3E55294014003020D77
:100E2000A4C1A330291C202B19E53B147006C2294C
:100E3000D22AA1A4F53BC3E55294014003020DA4BC
:100E40008061753C0078FA79A4E760027803C3E515
:100E50005398504FE523604B303A17203805203423
:100E600007800F303402800A202B07D22B855B5974
:100E7000A1D278F0302B05855B597820C3E54898DE
:100E80005003020DA4302B1BC22BC238303402D2C7
:100E900038D229753B12855B59A1A4053CE5526007
:100EA00002C1A6753C00C2AF11EC75240075250087
:100EB000D2AF1202ED11EC78A4E66006D287D2918F
:100EC000D293C3E53C94044002617081DF901A0D17
:100ED0007820F140E520B4550AA3F140E520B4AAFA
:100EE00002800611FFF107801D901A0378807B0AAB
:100EF000F140A308DBFA901A0F788C7B1AF140A31B
:100F000008DBFA901A2922C2AFF17FF159901A003A
:100F10007410F145A37401F145A37420F145901AB2
:100F20000378807B0AF144A308DBFA901A0F788CCF
:100F30007B1AF144A308DBFAF192F170901A29228E
:100F4000E493F622E6438F01538FFD75EF0275B7E8
:100F5000A575B7F1F0538FFE22438F02438F0175C1
:100F6000EF0275B7A575B7F1901A0DF0538FFC22FB
:100F7000901A0D7455F145901A0E74AAF145227A13
:100F80003079D07820901A40F140E520F709A3DAB3
:100F9000F7227A3079D0901A40E7F14509A3DAF9BF
:100FA000227C051202F1DCFB22C2AF120300120305
:100FB0000612030C1203121202E5120300120306BA
:100FC00012030C1203121202E5120300120306129E
:100FD000030C120312D2AF22C2AF12031212030C7F
:100FE0001203061203001202E512031212030C127E
:100FF00003061203001202E512031212030C12037D
:0710000006120300D2AF222B
:1019FD00020AE8100120FFFFFFFFFFFF09FF01FFB3
:101A0D0055AA01FFFFFFFFFF03FFFFFF25D0285061
:0D1A1D0004FF02FF7AFF0101FFFF0000FF40
:101A400023435F4C5F3230232020202020202020A1
:101A500023424C48454C492445464D3842313023B9
:101A60002020202020202020202020202020202076
:101C0000C2AFC2D37597DE7597AD7581C075A90057
:101C100043FF80752438752503B1C875EF0243F181
:101C20000153A4FED28075D4FF75E3407DFA78039A
:101C300079E67C10752200752300901DD57B067512
:101C400024987525013080028145208008D8FBD971
:101C5000F9DCF781B7308008D8FBD9F9DCF781B718
:101C6000B188E493A3C39A6004DDC381B7DBDBB121
:101C70007A6002812E7B08E493FAA3B15BDBF87AE9
:101C800030B15B752200752300B17AEAFCEBFDC32D
:101C9000ED94FE400EB17A8A278B28ED30E0048A5D
:101CA000828B83B17A7AC270D8C3ED94FE601350F0
:101CB000CEBD0023EC60097520007521FF020000F5
:101CC0008100A827A9280809D804D90281D4B17EA7
:101CD000EAF281C80D81A3C3ED94035047EDA2E061
:101CE00092007AC5C3E5829400E583941C5092204B
:101CF0000010438F02438F0175B7A575B7F1F0301F
:101D0000001DA827A9280809438F01538FFDD80477
:101D1000D902A11FE275B7A575B7F1F0A3A10E53C3
:101D20008FFC817F7AC1BD030CE493A3FAB13FDC41
:101D3000F8B137817F8181AA22AB23B15BEBFAEA4C
:101D40006222752608C3E52313F523E52213F52245
:101D500050066323A0632201D526EAB1C8B1C87535
:101D6000260AEAF4200102D280300102C280B1C802
:101D7000C3134002C201D526EB22B17EEAFB2080CC
:101D800002A17E308002A183752608AE24AF25C350
:101D9000EF13FFEE13FEB1CCB1C8C3EA13308002DB
:101DA0004480FA30E703632201C3E52313F523E5FA
:101DB0002213F52250066323A0632201D526D9E51C
:101DC0002265236523F52222AE24AF250E0FDEFE09
:101DD000DFFCD20122424C48656C6934373163E83C
:031DE000B1060148
:00000001FF
